:10000000F62EFF3FFF3FFF3F6E3003138312DA00EF
:100010007530DB006C30DC006C30DD00DE01A501EA
:10002000A601A301A4015708F0005808F100D70A5F
:100030000319D80A7008A2007108A1000A08A000DC
:100040008A1574208A11F00020088A007008AB001D
:1000500070080319282D2B08253A0319382856084B
:1000600084002B088000D60AA50A0319A60A1328C3
:10007000A701A801A301A4015708E5005808E6005C
:1000800031267008D7007108D8005708A200580818
:10009000A1000A08A0008A1574208A11F000200827
:1000A0008A000030F1007008E5008A1544208A11AA
:1000B000700803199B28A701A8012708F000280849
:1000C000F1000A30F4000030F500AC265708A20019
:1000D0005808A1000A08A0008A1574208A11E200BD
:1000E00020088A0062087007A70071080318013F02
:1000F000A8000030E21BFF30A8073030A702031C25
:10010000A803D70A0319D80A5708A2005808A10063
:100110000A08A0008A1574208A11F00020088A00BD
:100120000030F1007008E5008A1544208A1170083B
:10013000031D5D28C3285708A2005808A1000A081B
:10014000A0008A1574208A11E20020088A00620843
:100150002A3A031DC328590884000008F0007008DB
:1001600084000008A700840A0008A8005908840039
:100170000008F0000230F007590884007008800081
:10018000D70A0319D80A5708A2005808A1000A087C
:10019000A0008A1574208A11E20020088A006208F3
:1001A0002E3A031D4029D70A0319D80A5708A2007E
:1001B0005808A1000A08A0008A1574208A11E200DC
:1001C00020088A0062082A3A031DFF285908840083
:1001D0000008F000700884000008A900840A0008E4
:1001E000AA00590884000008F0000230F0075908FE
:1001F000840070088000D70A0319D80A3F29A90192
:10020000AA015708A2005808A1000A08A0008A15F0
:1002100074208A11F00020088A000030F100700874
:10022000E5008A1544208A11700803193F2929081E
:10023000F0002A08F1000A30F4000030F500AC2686
:100240005708A2005808A1000A08A0008A157420C7
:100250008A11E20020088A0062087007A90071086C
:100260000318013FAA000030E21BFF30AA0730301C
:10027000A902031CAA03D70A0319D80A0129422993
:10028000A901AA015708F0005808F100D70A03197C
:10029000D80A7008A2007108A1000A08A0008A15F7
:1002A00074208A11AB0020088A000E2A2508F0006D
:1002B0002608F100080023173B2A3B2AA316A317A0
:1002C0003B2A590884000008F000700884000008E8
:1002D000DF00590884000008F000F00A5908840083
:1002E000700880005F08003A031D78295A30DF004B
:1002F000E001E10160085F0784000008F000700879
:1003000003198629E00A0319E10A7A2929082A042F
:100310000319962961082A02031D90296008290201
:10032000031896292908E0002A08E100280861023C
:10033000031D9C29270860020318A5296008A7024D
:10034000031CA8036108A802A729A701A801A319F3
:10035000BE292708F0002808F1000130A702031C7D
:10036000A803700871040319BE29560884002030C0
:100370008000D60AA50A0319A60AA9296008F00078
:100380006108F1000130E002031CE1037008710410
:100390000319D8295F0884000008F000560884007B
:1003A00070088000D60ADF0AA50A0319A60ABE292A
:1003B000A31DEF292708F0002808F1000130A7024B
:1003C000031CA803700871040319EF295608840060
:1003D00020308000D60AA50A0319A60ADA291328B4
:1003E000590884000008F000700884000008AB0081
:1003F000590884000008F0000230F0075908840012
:10040000700880002B30DF000130E0000030E10098
:100410008629C030A3040030A4043B2A2B08003AEC
:10042000031956292B086C3A03195B292B086F3ADC
:1004300003195B292B08643A03195D292B08693AD3
:1004400003195D292B08703A03195E292B08583AC5
:1004500003195E292B08783A03195F292B08733A90
:10046000031961292B08633A0319F0292B08753AFF
:100470000319092A022AC0302305E2002408E300F8
:100480000030E30500306306031D482A0030620691
:10049000031D7B2A590884000008F00070088400BE
:1004A0000008DF00840A0008E00059088400000802
:1004B000F0000230F0075908840070088000803096
:1004C0006006F00080307002031D682A00305F0271
:1004D00003187A2A0330A3040030A4045F08003C08
:1004E000F0006008031C013FF101F1027008DF0019
:1004F0007108E000902A590884000008F000700894
:1005000084000008DF00840A0008E0005908840025
:100510000008F0000230F0075908840070088000DD
:1005200000302A06031D962A00302906031DA32A3F
:1005300000306006031D9E2A00305F06031DA32ABB
:10054000A90A0319AA0AC0302305F0007008E400C4
:10055000542B0130AB002B08053A0319E12A013076
:10056000F4002B08F000F10174080319BC2AF00D07
:10057000F10D7010FF3FB52A6030F0070830031806
:10058000013FF1077008A2007108A1000A08A0004D
:100590008A1574208A11E20020088A00A20A031931
:1005A000A10A8A1574208A11E30020088A006308D2
:1005B0006002031DDD2A62085F02031CE12AAB0A08
:1005C000AB2A642B0130AB002B08043A03191A2B19
:1005D0000130F4002B08F000F10174080319F52A2A
:1005E000F00DF10D7010FF3FEE2A6B30F007083070
:1005F0000318013FF1077008A2007108A1000A0862
:10060000A0008A1574208A11E20020088A00A20A3C
:100610000319A10A8A1574208A11E30020088A00B0
:1006200063086002031D162B62085F02031C1A2B6D
:10063000AB0AE42A642B0130AB002B08063A0319FD
:10064000532B0130F4002B08F000F101740803195A
:100650002E2BF00DF10D7010FF3F272B5330F007BC
:1006600008300318013FF1077008A2007108A100CB
:100670000A08A0008A1574208A11E20020088A0066
:10068000A20A0319A10A8A1574208A11E30020081E
:100690008A0063086002031D4F2B62085F02031C7F
:1006A000532BAB0A1D2B642B6408003A0319A92AAB
:1006B0006408C03A0319A92A6408803A0319E22A97
:1006C0006408403A03191B2B8030F00080302A0662
:1006D0007002031D6D2B29082B020318722B2908A9
:1006E000AB00802B80302A06F00080307002031DA2
:1006F0007B2B2B0829020318802B2B08A900AA01A9
:10070000270828040319932B03302305F00024083D
:10071000F1000030F105700871040319932B0130CA
:10072000A702031CA80380302A06F00080302806A8
:100730007002031D9D2B270829020318A62B2908E8
:10074000A702031CA8032A08A802A82BA701A80136
:10075000C4302305E20024080839E3006308083A9E
:10076000031DB42B40306206031DBF2B270828044D
:100770000319BE2B0130A702031CA803DF2BC030D6
:100780002305E20024080839E3006308083A031D42
:10079000CB2B80306206031DDF2B8030F0008030D1
:1007A00028067002031DD62B2708023C0318DD2BF8
:1007B0000230A702031CA803DF2BA701A8015608DB
:1007C000E5002D257008D6002908F0002A08F10060
:1007D0000130A902031CAA037008710403190A2D31
:1007E000C0302305F0007008E200F12C0130F40065
:1007F0002908F0002A08F10074080319042CF00DF0
:10080000F10D7010FF3FFD2B6030F007083003182A
:10081000013FF1077008A2007108A1000A08A000BA
:100820008A1574208A11F40020088A00A20A03198C
:10083000A10A8A1574208A11F50020088A005F0831
:10084000F0006008F1004D270A30F4000030F50098
:100850004D277808F0007908F10030307007AB00C0
:10086000012DA31E782C0130F4002908F0002A087D
:10087000F10074080319412CF00DF10D7010FF3FC9
:100880003A2C6B30F00708300318013FF10770086D
:10089000A2007108A1000A08A0008A1574208A111C
:1008A000F40020088A00A20A0319A10A8A157420FC
:1008B0008A11F50020088A005F08F0006008F10046
:1008C0004D270F30F0050030F1051230F0070830E9
:1008D0000318013FF1077008A2007108A1000A087F
:1008E000A0008A1574208A11AB0020088A00BC2C55
:1008F0000130F4002908F0002A08F10074080319F7
:10090000862CF00DF10D7010FF3F7F2C6B30F0073F
:1009100008300318013FF1077008A2007108A10018
:100920000A08A0008A1574208A11F40020088A00A1
:10093000A20A0319A10A8A1574208A11F500200859
:100940008A005F08F0006008F1004D270F30F005C5
:100950000030F1050030F00708300318013FF107BF
:100960007008A2007108A1000A08A0008A1574206E
:100970008A11AB0020088A00012D0130F4002908FB
:10098000F0002A08F10074080319CB2CF00DF10DCA
:100990007010FF3FC42C5330F00708300318013F9C
:1009A000F1077008A2007108A1000A08A0008A15CA
:1009B00074208A11F40020088A00A20A0319A10AEF
:1009C0008A1574208A11F50020088A005F08F0005B
:1009D0006008F1004D2707307005AB003030AB07E1
:1009E000012D6208003A0319F62B6208C03A031978
:1009F000F62B6208803A0319312C6208403A031939
:100A0000BD2C560884002B088000D60AA50A0319BD
:100A1000A60AE42BA31D272D8030F0008030280685
:100A20007002031D152D2708003C0318272D5608BA
:100A3000840020308000D60AA50A0319A60A0130D6
:100A4000A702031CA80327082804031D172D132839
:100A50002508F0002608F100080003138312231D67
:100A60009A2DA31C4C2D01302305F0002408F10021
:100A70000030F105700871040319412D2D30F0008C
:100A8000432D2B30F0006508840070088000E50AD3
:100A9000A50A0319A60A852D01302305F0002408B4
:100AA000F1000030F105700871040319602D65082C
:100AB000840020308000E50AA50A0319A60A852DC6
:100AC000C0302305F20024080839F3007308083AFF
:100AD000031D6C2D80307206031D852D6508840072
:100AE00030308000E50AA50A0319A60AA31E7B2D53
:100AF0005830F0007D2D7830F000650884007008D3
:100B00008000E50AA50A0319A60A27082804031984
:100B1000992D6508840030308000E50AA50A031984
:100B2000A60A0130A702031CA80327082804031DF6
:100B3000892D1A2E270828040319B02DA319B02DCA
:100B40006508840020308000E50AA50A0319A60A7A
:100B50000130A702031CA80327082804031DA02DA9
:100B6000A31CCB2D01302305F0002408F100003038
:100B7000F105700871040319C02D2D30F000C22D4D
:100B80002B30F0006508840070088000E50AA50A93
:100B90000319A60ADE2D01302305F0002408F10018
:100BA0000030F105700871040319DE2D650884001A
:100BB00020308000E50AA50A0319A60AC0302305E3
:100BC000F20024080839F3007308083A031DEA2DDF
:100BD00040307206031DF52D65088400303080001A
:100BE000E50AA50A0319A60A1A2EC0302305F20049
:100BF00024080839F3007308083A031D012E8030D9
:100C00007206031D1A2E6508840030308000E50A44
:100C1000A50A0319A60AA31E102E5830F000122EA2
:100C20007830F0006508840070088000E50AA50AA5
:100C30000319A60A8030F00080302A067002031DD6
:100C4000232E29082B0203182E2E6508840030302D
:100C50008000E50AA50A0319A60A1A2E6508F00005
:100C600008004D2E03138312A315E50A0319E60AA3
:100C7000A02E2314E50A0319E60AA02EA314E50A00
:100C80000319E60AA02EA415E50A0319E60AA02E08
:100C90002315E50A0319E60AA02E0313831265083B
:100CA000A2006608A1000A08A0008A1574208A1113
:100CB000F20020088A0072082D3A0319322E6508C6
:100CC000A2006608A1000A08A0008A1574208A11F3
:100CD000F20020088A007208203A0319392E6508AC
:100CE000A2006608A1000A08A0008A1574208A11D3
:100CF000F20020088A0072082B3A03193E2E65087C
:100D0000A2006608A1000A08A0008A1574208A11B2
:100D1000F20020088A007208233A0319432E65085E
:100D2000A2006608A1000A08A0008A1574208A1192
:100D3000F20020088A007208303A0319482EA12ECA
:100D4000312EA31CA42E2310A31DA72E231165084A
:100D5000F0006608F100080003138312FB01FA019A
:100D6000F9018030F800FD01F11FBC2EF109F009F6
:100D7000F00A0319F10AFD0AF51FC42EF509F4095A
:100D8000F40A0319F50AFD0AF10CF00C031CD12E2C
:100D90007408F90775080318750FFA070318FB0A9A
:100DA0000310F01FD92E7408FA070318FB0A750800
:100DB000FB07FB0CFA0CF90CF80C031CC42E7D1C71
:100DC000EC2EFB09FA09F909F809F80A0319F90ADE
:100DD0000319FA0A0319FB0A7B08F3007A08F200E8
:100DE0007908F1007808F000000008008A157B20DF
:100DF0008A1119308316990018158A1524208A1132
:100E00002E30CE008230CF000830D0002C08D10028
:100E10002D08D2003227AC0A0319AD0A2E30CE00BD
:100E20006A270330FC00FF30FB00FF30FA00FC0BA8
:100E30001A2F212FFB0B1D2F202FFA0B1D2F1A2FDE
:100E4000172F8C30FB00FF30FA00FB0B282F2B2FC5
:100E5000FA0B282F252FA130FA00FA0B2D2F0000B6
:100E6000002F312F513003138312D5004E08D600C6
:100E70004F08D7005008D8005530D900042070081A
:100E8000D3007108D4004E08F00770088400800178
:100E90005308F0005408F100080003138312F8010E
:100EA000F9011030FC00710DF80DF90D7408F8020D
:100EB0007508031C750FF9020318652F7408F807ED
:100EC00075080318750FF9070310F00DF10DFC0BF1
:100ED000532F080003138312CF014F084E078400DD
:100EE0000008F1007108003A0319802F4F084E07DF
:100EF00084000008D6008A1534208A11CF0A6D2F8D
:100F00004E08F0000800FF3FFF3FFF3FFF3FFF3F5D
:100F1000FF3FFF3FFF3FFF3FFF3FFF3FFF3FFF3FE1
:100F2000FF3FFF3FFF3FFF3FFF3FFF3FFF3FFF3FD1
:100F3000FF3FFF3FFF3FFF3FFF3FFF3FFF3FFF3FC1
:100F4000FF3FFF3FFF3FFF3FFF3FFF3FFF3FFF3FB1
:100F5000FF3FFF3FFF3FFF3FFF3FFF3FFF3FFF3FA1
:100F6000FF3FFF3FFF3FFF3FFF3FFF3FFF3FFF3F91
:100F7000FF3FFF3FFF3FFF3FFF3FFF3FFF3FFF3F81
:100F8000FF3FFF3FFF3FFF3FFF3FFF3FFF3FFF3F71
:100F9000FF3FFF3FFF3FFF3FFF3FFF3FFF3FFF3F61
:100FA000FF3FFF3FFF3FFF3FFF3FFF3FFF3FFF3F51
:100FB000FF3FFF3FFF3FFF3FFF3FFF3FFF3FFF3F41
:100FC000FF3FFF3FFF3FFF3FFF3FFF3FFF3FFF3F31
:100FD000FF3FFF3FFF3FFF3FFF3FFF3FFF3FFF3F21
:100FE000FF3FFF3FFF3FFF3FFF3FFF3FFF3FFF3F11
:100FF000FF3FFF3FFF3FFF3FFF3FFF3FFF3FFF3F01
:1010000030343134323433343434353436343734A4
:10101000383439346134623463346434653466346A
:10102000003408003034313432343334343435341D
:101030003634373438343934413442344334443428
:101040004534463400340800031383169816903054
:101050008312980083168717071383128C1E332878
:101060001A08D2002D2808000030031383169818A0
:101070000130F1007108003A031D402800003428B7
:101080008312560899000800031383126508393C3F
:10109000031C512830306502031C51280130F00038
:1010A0005228F00108000134003408340034403480
:1010B000003400340234003410340034803408002A
:1010C000013400340A34003464340034E834033426
:1010D0001034273408000134003410340034003454
:1010E00001340034103408000313831221088A00ED
:1010F000220882000800003003138312AC00003085
:10110000AD0008000D340A3425346434003408007E
:04400E00D52FFFFFAC
:00000001FF
